:020000040000FA
:020000002028B6
:080008008F00030803138312AB
:100010008E0004088C000A088D008A010B19112833
:1000200017280B11FB3081001408031D94030D08E1
:100030008A000C0884000E0883008F0E0F0E090042
:10004000DC20920A05301202031D28289201212883
:1000500012086920860006080F39F13E031921288D
:10006000AC200F39F13E03192128BC208D2003302C
:1000700091005730D720910B39282128E535F03CE5
:10008000E4306117ED392D1024106529693BE939F9
:10009000EE37201DAE18B41924102D104310F03780
:1000A000F23CE7347434321030182C195410EE3A04
:1000B0007232D730F230A032EE24AE312016EC206E
:1000C00020366929E833733A5210F332F232653B35
:1000D0002E328207F034E034D034B03470348207EA
:1000E0000134043407340E348207023405340834F2
:1000F000003482070334063409340F3482070A348B
:100100000B340C340D3482070034003401340034D5
:100110000234003400340034033400301007031973
:1001200098281308850005160130D720051208000D
:10013000043091000510131C9E280514851401300D
:10014000D720851091030319A728930C9A28051529
:100150000130D720051108000608930005309100F2
:100160000A30D720060893020319B8289300AE2856
:100170009300910BB028080013090F3983209300D6
:100180001208FF3E8207C728CB28CF28D3281308A0
:100190006F209300080013087420930008001308D0
:1001A00079209300080013087E2093000800940033
:1001B0001408031DD82808008B019001051A900926
:1001C0008316E030850083160F30860081010430ED
:1001D00081048312FB308100850186019201930125
:0A01E000910194018B168B170800A3
:084000000100020003000400AE
:02400E00F33F7E
:00000001FF
